:020000040000FA
:020000008F2847
:080008008B13A300030EA400FA
:100010000C1C4828D0308F000508BD0004392C0680
:10002000031D2028A80B2A282C08AB00043A031D26
:100030001B2885161C2885122708A800A9002A2835
:100040008400AC06A90B282885122B112708A900CB
:100050002708A8003D0808393C06031D3D28B80BB9
:1000600047283C08BB00083A031D382805163928E4
:1000700005123708B800B90047288800BC06B90B3C
:1000800045280512BB113708B9003708B8000C1015
:100090000B1D55288B1E532825088100851C5228CE
:1000A0008510532885140B115528240E8300A30EA8
:1000B000230E8B1709008316413081000D30850017
:1000C00010309F000C14FF2390008312073099001A
:1000D00085108511013090008B160B178B170800C7
:1000E0004E30A5000030A6000030A6000030AC0065
:1000F000AB001030A700A800A9000030BC00BB0076
:100100001030B700B800B9000800A20B852808001D
:1001100085160A30852085120A30852088285B20C4
:100120007020051896288B1226109C2826189C28CB
:0A0130002614250881008B16912883
:00000001FF
